:100000000C9441000C945E000C945E000C945E0015
:100010000C945E000C945E000C945E000C945E00E8
:100020000C945E000C945E000C945E000C9418031B
:100030000C945E000C945E000C945E000C945E00C8
:100040000C945E000C945E000C94B5000C945E0061
:100050000C945E000C9460000C945E000C945E00A6
:100060000C945E000C945E00244750524D430024D3
:100070004750474741002E6C6F6700244750524D50
:10008000430011241FBECFEFD4E0DEBFCDBF11E08F
:10009000A0E0B1E0E8E2FAE202C005900D92AC30D7
:1000A000B107D9F714E0ACE0B1E001C01D92AD3466
:1000B000B107E1F70E9435010C9412150C94000071
:1000C0001F920F920FB60F9211242F933F938F938D
:1000D000209178003091790080917C00203D31059D
:1000E00070F480910F018F3030F080916F0181604A
:1000F00080936F0106C08F5F80930F0102C0109242
:100100000F0181E02C32380770F080910E018F30A2
:1001100030F080916F018E7F80936F0106C08F5FFA
:1001200080930E0102C010920E013093750120934E
:10013000740182E480937C0080917C0030931002F3
:1001400020930F0281E480937C008FED80937A00EE
:100150008F913F912F910F900FBE0F901F90189588
:1001600060E070E081EA96E308951F920F920FB667
:100170000F9211248F939F93EF93FF939091C6005A
:1001800080917801863988F48F5F8093780180911F
:100190007601E82FF0E0EA58FE4F93838F5F8639AF
:1001A00008F080E08093760105C080916F01826045
:1001B00080936F01FF91EF919F918F910F900FBEF0
:1001C0000F901F90189590E051E448E901C090E02D
:1001D00080916F0180FD46C0309177018091780158
:1001E000882311F420E013C0E32FF0E0EA58FE4F1B
:1001F0002381E32FEF5FF894809178018150809301
:1002000078017894E63908F0E0E0E0937701809196
:100210006F0181FF14C0F8941092C1001092770111
:1002200010927601109278015093C4004093C1005F
:1002300080916F018D7F80936F017894C8CF2223C6
:1002400039F2992319F4243209F0C2CFE92FF0E0F2
:10025000E35EFE4F20839F5F2A3029F0923508F03D
:10026000B6CFB6CF90E0892F0895A2E0B0E0EBE3DF
:10027000F1E00C94C7148DE085B98EE284B98FE368
:1002800088B917B88EEA8BB982E58AB980E58CBD4A
:1002900081E08DBD83ED90E3909389008093880089
:1002A0008AE08093810082E080936F0082E187BDC5
:1002B00082E484BD81E480937C008FED80937A009A
:1002C00078946DE272E080E00E947F09EE24FF24C2
:1002D00053E0A52E45E0B42E3DE1C32E31E0D32EF0
:1002E0004E010894811C911C28E1222E21E0322E1F
:1002F00090E7692E91E0792E80E0482E81E0582E1B
:100300001092C100299884E680931C0194E68091A4
:100310006F0180FF02C090931C0180911C01882313
:10032000B1F7299A8FEF80931C011FEF80916F0125
:1003300080FD05C080E00E94950F81FF02C01093F0
:100340001C0180911C01882389F791E00EC0A5BC97
:10035000B0921C0180911C018823E1F715BCB0927A
:100360001C0180911C018823E1F7915080F7F894DB
:100370001092C100109277011092760110927801CC
:1003800081E48093C40088E98093C10080916F016B
:100390008D7F80936F01789402C0EE24FF240E9429
:1003A000E300882309F4ACCF2BE730E0ADE1B1E006
:1003B000F9012F5F3F4F9491992329F08C91981761
:1003C00071F41196F5CFEDE1F1E082E09081913288
:1003D00020F331969C32D1F78150C1F77F01E114AF
:1003E000F104E9F2F70180818134C9F6EDE1F1E031
:1003F00089E09081913208F4F0C031969C32C9F7BF
:100400008150B9F77F01309709F4E7C08481958165
:1004100090931E0180931D0182819381909320010E
:1004200080931F018081918190932201809321010B
:1004300066E770E083E291E00E948F1142E16DE196
:1004400071E081E192E00E94D709892B09F0C7C0D1
:1004500040911B0250911C0260911D0270911E027E
:1004600081E192E00E943C05892B09F0B8C092E03E
:100470000EC0A5BCB0921C0180911C018823E1F73D
:1004800015BCB0921C0180911C018823E1F79150AA
:1004900080F785C02FE630E0ADE1B1E0F9012F5FD4
:1004A0003F4F9491992389F08C91981709F0AEC031
:1004B0001196F4CF1196F9012F5F3F4F9491992334
:1004C00021F08C919817B1F357C0042F10E09401DC
:1004D000A8016DE171E081E192E00E940E07892B95
:1004E00009F064C089819A810817190709F05EC074
:1004F0004AE050E068E171E08091740190917501EB
:100500000E94B3114AE050E060E771E080910F0271
:10051000909110020E94B3117F926F923F922F929E
:100520005F924F92DF92CF920E94D411F601019018
:100530000020E9F73197EC19FD099401AF016DE155
:1005400071E081E192E00E940E072DB73EB7285F6F
:100550003F4F0FB6F8943EBF0FBE2DBF892B41F51C
:10056000D6010D900020E9F71197AC19BD098981DA
:100570009A81A817B907E1F480916F0182FF0FC03B
:1005800081E192E00E94A906892B11F096E028C033
:10059000F89480916F018B7F80936F0178940E9413
:1005A000E300482F882309F075CF35C095E018C0C7
:1005B00098E016C0A5BC32E330931C0180911C0169
:1005C0008823E1F715BC82E380931C0180911C0114
:1005D0008823E1F7915070F793CE93E001C094E047
:1005E0001092C100299833E029E135BD20931C0108
:1005F00080911C018823E1F715BC20931C01809198
:100600001C018823E1F7915081F7FFCF28E630E005
:10061000ADE1B1E050CF1092C100299881E192E0A4
:100620000E940007892B11F097E0DACF91E0D2CF3A
:100630001F920F920FB60F9211242F938F939F93B7
:1006400080911C01882319F0815080931C018091B6
:100650000C0190910D01019690930D0180930C0176
:100660008055964448F010920D0110920C01809133
:100670006F01846080936F010E946F119F918F9131
:100680002F910F900FBE0F901F901895FC010097AF
:1006900069F0808191818617970741F480E00E947C
:1006A000950F282F30E02170307002C02CE030E030
:1006B000C9010895A0E0B0E0E0E6F3E00C94CB14AB
:1006C0004B015C01C0911001D0911101CC80DD8003
:1006D000EE80FF80C616D706E806F90609F44EC07C
:1006E0008F8D8823A1F180E2682E712C6C0E7D1E07
:1006F00001E0A7019601B30180E00E94FB0F892B66
:10070000D9F51F8E8C899D89A0E0B0E028853985B8
:100710004A855B85820F931FA41FB51FC816D90693
:10072000EA06FB06A0F41E8D10C08C899D89A0E00E
:10073000B0E0C80ED91EEA1EFB1E01E0A70196011B
:10074000B30180E00E94FB0F1150123070F781144A
:100750009104A104B10491F0BE01605E7F4F01E0FD
:10076000A501940180E00E949C0F892B29F48C82C2
:100770009D82AE82BF8202C080E001C081E0CDB721
:10078000DEB7EEE00C94E714A0E0B0E0EAECF3E0B2
:100790000C94CB14EC014B01E0901001F09011018E
:1007A000F701A084B184C284D384848D813021F088
:1007B000823009F072C05AC08E01000F111F0C0F59
:1007C0001D1F16950795B801672F7727669580E05E
:1007D00090E06A0D7B1D8C1D9D1D0E945A0388238D
:1007E00009F45BC0D801B17051E0652E712C6C2208
:1007F0007D22C0FF0AC0F701EA0FFB1F80A18F70A6
:10080000982D9295907F982B01C0982DAE0DBF1D0D
:10081000FD0190A3E801219681E0F701878FBE01D9
:10082000672F7727669580E090E06A0D7B1D8C1D11
:100830009D1D0E945A03882381F1DE01B17061146D
:10084000710439F034E0969487943A95E1F7982D45
:1008500008C0F701EA0FFB1F90A1907F892D8F70D0
:10086000982BAE0DBF1DFD0190A313C06D2F7727F0
:1008700080E090E06A0D7B1D8C1D9D1D0E945A0337
:10088000882359F0CC0FDD1FD170CE0DDF1D99A24A
:1008900088A281E0F701878F01C080E0CDB7DEB785
:1008A000EEE00C94E714A0E0B0E0E9E5F4E00C948D
:1008B000CE148C01E0901001F0901101823091056E
:1008C00008F467C0E7018E899F890817190708F0A7
:1008D00060C0A884B984CA84DB848C8D813021F007
:1008E000823009F056C040C0E801CC0FDD1FC00FB8
:1008F000D11FD695C795BE01672F7727669580E0F3
:1009000090E06A0D7B1D8C1D9D1D0E945A0388235B
:1009100009F43FC0FE01F170EE0DFF1D90A021967D
:10092000BE01672F7727669580E090E06A0D7B1DFA
:100930008C1D9D1D0E945A03882359F1292D30E0FA
:10094000D170EC0EFD1EF70190A180E0282B392B11
:1009500000FF07C0F90194E0F695E7959A95E1F755
:100960001AC0F901FF7017C0612F772780E090E06F
:100970006A0D7B1D8C1D9D1D0E945A03882349F022
:10098000000F111F1170E00EF11EE701E8A1F9A19F
:1009900002C0E1E0F0E0CF01CDB7DEB7EBE00C94B0
:1009A000EA14A0E0B0E0E7EDF4E00C94CF147C0191
:1009B000C0901001D0901101F601A688B788009769
:1009C00049F4008D118D0230110588F00A151B05C0
:1009D00070F40FC00E9453049C018230910508F40A
:1009E00040C08A159B0508F441C0870102C001E0A0
:1009F00010E0E8012196CA15DB0528F00230110548
:100A000098F1C2E0D0E0CE010E9453049C0100970F
:100A100039F08130910551F1C017D10759F724C041
:100A20001C2F0D2F6FEF7FEFCE010E94C403882390
:100A3000C1F0E114F10431F0BE01C7010E94C4030A
:100A4000882379F0F601108F018F828D938DFFEF4F
:100A50008F3F9F0721F00197F601938F828F9E01B0
:100A600005C021E030E002C020E030E0C901CDB790
:100A7000DEB7EAE00C94EB14A0E0B0E0E2E4F5E0CD
:100A80000C94CB14EC017A018B016C807D80688121
:100A90007981C3010E9446034C01009709F0D6C03A
:100AA0008A8187FDD0C0AA84BB84CC84DD84AE1447
:100AB000BF04C006D10610F481FF02C057016801CF
:100AC0001E821F821886198681E08B83A114B104CF
:100AD000C104D10409F49DC06E857F85611571053F
:100AE00071F480E090E00E94D104BC018130910556
:100AF00009F4A6C09F878E87009709F48AC0F30186
:100B0000858DE82EFF2400E010E0F9E0EE0CFF1CDC
:100B1000001F111FFA95D1F7798B688BEA14FB043B
:100B20000C051D0558F58A8181FF04C0CB010E9488
:100B3000D10403C0CB010E945304BC010097E1F033
:100B40008130910509F47CC0F30186899789681783
:100B5000790708F075C08E819F81A885B9858E0DB3
:100B60009F1DA01FB11F8E839F83A887B987AE18D2
:100B7000BF08C00AD10AD0CF57016801D601C5010C
:100B80000197A109B109E9E0B695A79597958795D1
:100B9000EA95D1F7F82E00911001109111016250E1
:100BA0007040F8018689978902976817790728F0BD
:100BB00020E030E040E050E014C080E090E0F80138
:100BC000258D30E040E050E00E9486149B01AC018E
:100BD000F80180899189A289B389280F391F4A1F9A
:100BE0005B1F2F0D311D411D511D2A8B3B8B4C8BE3
:100BF0005D8BF301858D8F198B838E819F81A885F5
:100C0000B9858A0D9B1DAC1DBD1D8E839F83A88752
:100C1000B9876A8161FF1AC02E813F814885598555
:100C20008A859B85AC85BD8582179307A407B50788
:100C300068F42A873B874C875D8760626A8306C0B9
:100C40008A8180688A8368E0862E912CC401CDB7A2
:100C5000DEB7EEE00C94E714EF92FF920F931F9330
:100C6000CF93DF938C01C0911001D0911101FC0151
:100C7000E280F3800894E11CF11CC7018F70907032
:100C8000892B09F05BC082859385A485B585019683
:100C9000A11DB11D82879387A487B58740855185A3
:100CA0004115510539F48A819B81E816F90608F44B
:100CB00045C049C08D8D90E001979701A4E036951D
:100CC0002795AA95E1F782239323892BB9F5CA01C9
:100CD0000E945304BC0182309105A8F18E899F893E
:100CE0006817790780F5F80171876087C091100156
:100CF000D0911101625070408E899F8902976817C8
:100D0000790728F020E030E040E050E012C080E0B9
:100D100090E02D8D30E040E050E00E9486149B0171
:100D2000AC0188899989AA89BB89280F391F4A1F74
:100D30005B1FF8012287338744875587F801F382C8
:100D4000E28281E001C080E0CDB7DEB7E6E00C943E
:100D5000EF14EF92FF920F931F93CF93DF93EC0169
:100D6000688179818C819D810E9446037C01009776
:100D700009F040C08A8185FF3DC06E897F89888DDA
:100D8000998D0E945A03882391F10A8D1B8DF801D9
:100D90008385806283878A859B85AC85BD85848FAA
:100DA000958FA68FB78F8E859F85938F828F0E9498
:100DB000B000F801668B778B808F918F8A818F7D51
:100DC0008A83E0911001F091110181E0878F60E04A
:100DD00070E080E090E00E945A03882341F040E0F8
:100DE00050E063E080E00E947710892B19F0B8E0B2
:100DF000EB2EF12CC701CDB7DEB7E6E00C94EF1473
:100E0000CF93DF93EC010E94A9069C01009711F497
:100E10001D821C82C901DF91CF910895A0E0B0E04E
:100E2000E4E1F7E00C94C814EC01162F072F7A01C7
:100E30003901AC80BD80F90111821082688179810D
:100E4000C5010E9446034C01009709F03BC18A810D
:100E500087FD35C181FD04C036E0832E912C32C15F
:100E60002A853B854C855D85C701A0E0B0E0820FF7
:100E7000931FA41FB51F82179307A407B50708F493
:100E800021C1812F902F9C016901412C22E0522E1B
:100E900033243394F8C02E813F8148855985DA0187
:100EA000C9019170A070B0700097A105B10509F05B
:100EB000B1C08B8181508B83882349F02A893B897B
:100EC0004C895D892F5F3F4F4F4F5F4F51C02115B8
:100ED00031054105510569F46E857F856115710500
:100EE00089F480E090E00E94D104BC019F878E8746
:100EF00005C0888999890E94D104BC0161157105DA
:100F000009F4C5C06130710509F4D6C0F5018689C0
:100F100097896817790708F0CFC0798B688B0091A3
:100F200010011091110162507040F8018689978973
:100F300002976817790728F020E030E040E050E0A1
:100F400014C080E090E0F801258D30E040E050E0F2
:100F50000E9486149B01AC01F80180899189A289C5
:100F6000B389280F391F4A1F5B1FF501858D8B83BD
:100F70002A8B3B8B4C8B5D8B0F2D069561F16B8122
:100F8000102F601708F4162F012FB60180E00E9481
:100F9000FB0F892B09F090C08B818F5F811B8B83A6
:100FA000812F90E001979C01442737FD4095542FF5
:100FB0008C010F5F1F4F8A899B89AC89BD89820F85
:100FC000931FA41FB51F8A8B9B8BAC8BBD8B102FDF
:100FD0000027110F3EC02E813F81488559858A85A3
:100FE0009B85AC85BD85281739074A075B0790F0BC
:100FF00060E070E080E090E00E945A03882309F4EA
:101000005BC08A899B89AC89BD89F50184839583FE
:10101000A683B7836A897B898C899D890E945A033C
:10102000882309F449C02E813F813170C201821B9F
:10103000930B87018E159F0508F48C01205E3F4FAE
:101040002A0D3B1DA801B601C9010E94A311F5019B
:10105000378EC00ED11EC801A0E0B0E02E813F81C6
:1010600048855985280F391F4A1F5B1F2E833F83F0
:1010700048875987F30180819181800F911F918367
:101080008083E01AF10AE114F10409F004CF2E8103
:101090003F81488559858A859B85AC85BD858217AA
:1010A0009307A407B50720F42A873B874C875D8701
:1010B0008A8180628A8306C08A8180688A8388E008
:1010C000882E912CC401CDB7DEB7E1E10C94E41475
:1010D000A0E0B0E0EEE6F8E00C94C914EC01162FA5
:1010E000072F7A0139018C809D80F90111821082CD
:1010F00068817981C4010E9446035C01009709F070
:10110000F8C08A8187FDF2C080FD04C076E0A72E7A
:10111000B12CEFC02A853B854C855D858E819F81F2
:10112000A885B985281B390B4A0B5B0BC701A0E0CA
:10113000B0E0281739074A075B0708F47901812FC7
:10114000902F9C016901412C62E0562EC7C02E8170
:101150003F8148855985DA01C9019170A070B0704E
:101160000097A105B10509F084C08B8181508B8364
:10117000882349F02A893B894C895D892F5F3F4F3D
:101180004F4F5F4F43C0211531054105510519F4FB
:101190006E857F8505C0888999890E945304BC01AA
:1011A0006230710508F49FC0F40186899789681739
:1011B000790708F098C0798B688B00911001109125
:1011C000110162507040F80186899789029768176B
:1011D000790728F020E030E040E050E014C080E0E3
:1011E00090E0F801258D30E040E050E00E94861448
:1011F0009B01AC01F80180899189A289B389280FEC
:10120000391F4A1F5B1FF401858D8B832A8B3B8B13
:101210004C8B5D8B0F2D069561F16B81102F601744
:1012200008F4162F012FB60180E00E949C0F892B35
:1012300009F059C08B818F5F811B8B83812F90E0D8
:1012400001979C01442737FD4095542F8C010F5F77
:101250001F4F8A899B89AC89BD89820F931FA41F68
:10126000B51F8A8B9B8BAC8BBD8B102F0027110F6A
:101270001BC06A897B898C899D890E945A038823B7
:1012800091F18E819F8191709201281B390B87010A
:101290002E153F0508F489018096880D991DA80137
:1012A000BC01C6010E94A311C00ED11EC801A0E05E
:1012B000B0E02E813F8148855985280F391F4A1F8C
:1012C0005B1F2E833F8348875987F301808191817B
:1012D000800F911F91838083E01AF10AE114F104D9
:1012E00009F035CF06C08A8180688A8348E0A42E41
:1012F000B12CC501CDB7DEB7E0E10C94E514CF9376
:10130000DF93FB01882319F025E030E01DC0A09198
:101310001001B091110170931101609310011097A9
:1013200041F080E292E0ED019C01199221503040A1
:10133000E1F7309739F080E292E0DF01EC011D9295
:101340002197E9F720E030E0C901DF91CF910895BE
:101350000F93CF93DF939B01AC01C0911001D0910B
:101360001101BE01605E7F4F01E080E00E949C0F92
:10137000892BC1F4C25EDD4F88819981CE51D24064
:1013800085559A4A79F443E050E067E071E0CE0178
:101390008A5A9F4F0E9496119C0180E0232B19F0DE
:1013A00081E001C082E0DF91CF910F910895ADE11E
:1013B000B0E0EDEDF9E00C94C7149D8F8C8F3B01EC
:1013C0008090100190901101FC011582148203C0DD
:1013D0000894611C711CF30180818032C9F38F3243
:1013E00019F40894611C711C8114910409F417C14B
:1013F000F42FFF71FB8F142F1E71F401848D88234D
:1014000059F080E00E94950F80FD06C0112309F479
:10141000ABC382FD07C1A8C380E292E0F4019C0146
:10142000119221503040E1F780E00E94B80E80FF19
:1014300003C021E030E08BC3112311F082FDF2C024
:1014400060E070E080E090E00E94A809813021F027
:10145000EE24FF2487011EC082EE91E0880E991EC3
:10146000F40180812EE13EEF820E931E882309F461
:10147000DCC086EE91E0880E991EF401E080F180D8
:10148000028113812AE13EEF820E931EC801B7014B
:101490000E94A809882309F0C8C0F40183A594A577
:1014A0008050924009F0C1C0F40186A997A9BC01FF
:1014B00080E090E0611571058105910569F424E4EF
:1014C00030E0820E931EF4016081718182819381EC
:1014D0002CEB3FEF820E931EF401758B648B20A9D9
:1014E000268F30E040E050E00E9486145B016C01E2
:1014F000F40186A597A5A0E0B0E0E80EF91E0A1F4A
:101500001B1FE086F1860287138785A5858F21A999
:1015100032A93383228383A994A97C0100E010E0DF
:10152000E114F1040105110569F480E490E0880EEE
:10153000991EF401E080F1800281138180EC9FEF1D
:10154000880E991EF40186A597A5A0E0B0E0E81AE0
:10155000F90A0A0B1B0BEA18FB080C091D09A4E089
:1015600036952795AA95E1F7C901A0E0B0E0E81A01
:10157000F90A0A0B1B0B258D30E040E050E0C80152
:10158000B7010E94A5142E5F3F4F4F4F5F4FF401EC
:10159000378B268B283FFFE03F07F0E04F07F0E056
:1015A0005F0710F461E006C0285F3F4F40405040A5
:1015B000E0F562E0F4012085318542855385D6014E
:1015C000C501820F931FA41FB51F84879587A68727
:1015D000B7878281938174E0969587957A95E1F734
:1015E000A0E0B0E0820F931FA41FB51F8A0D9B1DC2
:1015F000AC1DBD1D808B918BA28BB38B648F8FEF45
:101600009FEF938F828F8091120190911301019629
:10161000909313018093120191838083A5C22AE0E5
:1016200030E095C229E030E092C22BE030E08FC27A
:101630002E010894411C511C92E0292E312C4BE0C4
:1016400050E060E270E0C2010E94AC1120E048E08E
:1016500090E038E102C028E04BE0F30111913F0136
:10166000112311F01F3249F4222309F4C7C0392392
:101670003C87113009F044C0C1C0113208F4BEC02B
:101680001F3709F4BBC01E3241F490FDB7C02223BE
:1016900009F4B4C02930F8F2B1C0123209F4AEC076
:1016A0001A3220F11D3208F4A9C01A33F8F01034B0
:1016B00008F4A4C090FD1AC01C3709F49FC0812F04
:1016C0008B55833008F49AC0865E8A3128F44830FE
:1016D00011F4377F01C03F7E812F81568A3130F46B
:1016E0001052483011F4986001C09061241708F03E
:1016F00085C09E7FF201E20FF11D10832F5FADCFF9
:101700006F89788D898D9A8D0E945A03882331F4D0
:1017100090E09C01590128E030E084C02F85388991
:101720002F70307085E0220F331F8A95E1F7F601A4
:10173000E20FF31F80A18823E1F0853EA1F000E2D3
:10174000A02EB12CA20EB31EAC0CBD1CF5018385DE
:10175000082F83FD08C04BE050E0B201C5010E9494
:101760009611009751F0CE010D960E942C06882309
:1017700039F6112309F049C04FC0112319F420E0B4
:1017800030E050C004FF41C0F501E28CF38CFE8ACA
:10179000ED8A0091100110911101B7016250704063
:1017A000F8018689978902976817790728F020E061
:1017B00030E040E050E014C080E090E0F801258D7A
:1017C00030E040E050E00E9486149B01AC01F8013B
:1017D00080899189A289B389280F391F4A1F5B1F0D
:1017E000FC8AEB8A2F8B388F498F5A8F388A2F8645
:1017F00026CF20E030E0AA24BB2414C080E090E093
:101800009C01590124E030E00DC080E090E09C0193
:10181000590123E030E006C080E090E09C015901CE
:1018200022E030E0FB8D4F2F50E0CA018C719070A8
:10183000892B09F441C12115310509F4D6C02230A4
:10184000310509F084C160901001709011010B897D
:101850001C890115110551F11E8B0D8BB8016250C9
:101860007040F3018689978902976817790728F0F5
:1018700020E030E040E050E014C080E090E0F30170
:10188000258D30E040E050E00E9486149B01AC01C1
:10189000F30180899189A289B389280F391F4A1FD2
:1018A0005B1F2F8B388F498F5A8F09C0F3018485B6
:1018B0009585A685B7858F8B988FA98FBA8F188A43
:1018C0001F86BDE0EB2EF12CEC0EFD1E6F89788D8E
:1018D000898D9A8D0E945A03882309F433C1EF85BC
:1018E000F889EF70F070A5E0EE0FFF1FAA95E1F701
:1018F000B0965301AE0EBF1EB097E60DF71D80A146
:10190000882309F44CC1853E09F449C1C7010E94EE
:101910002C068823D9F60115110509F410C18D890B
:101920009E890E94D1048C01009709F408C181307E
:10193000910509F407C160E070E080E090E00E944A
:101940005A03882309F4FEC0A0901001B090110141
:10195000B80162507040F50186899789029768172F
:10196000790720F0CC24DD24760114C080E090E0DB
:10197000F501258D30E040E050E00E9486146B01B7
:101980007C01F50180899189A289B389C80ED91E8D
:10199000EA1EFB1EF301C482D582E682F782E0E2F2
:1019A000AE2EB12CA60CB71C80E092E0F5019C0194
:1019B000119221503040E1F7F301158D10C001E084
:1019C000A7019601B50180E00E94FB0F892B09F069
:1019D000B9C00894C11CD11CE11CF11C1150112389
:1019E00071F781E0F301878FDAC0F2FF03C027E0CF
:1019F00030E0ADC0A114B10409F4A1C0F5018385A4
:101A0000817109F09CC043FF42C0C28CD38C138EFD
:101A1000128E148E158E168E178E81E0F401878F2C
:101A20002480358046805780E0901001F0901101AD
:101A300086011CC0C8010E9453043C0181309105FD
:101A400009F480C060E070E0C8010E94C4038823EC
:101A500009F478C0F701828D938DFFEF8F3F9F07C8
:101A600021F00196F701938F828F830102301105D7
:101A700008F472C0F7018689978908171907D0F210
:101A80006BC00894C108D108F401D18EC08EFB8DC3
:101A9000F3FF22C080E2F50183870E94B000F501C8
:101AA000668B778B808F918F66877787808B918B02
:101AB00081E0F401878F10C02115310509F047C07E
:101AC000A114B10409F441C0F501838584FD3DC032
:101AD00041FF02C080FD33C0F40184819581A6815D
:101AE000B781EC8DFD8D868B978BA08FB18FB38ED8
:101AF000A28E2B8D2283F501828D938DEC8DFD8D31
:101B000097878687F501848D958DA68DB78DEC8D91
:101B1000FD8D82879387A487B587168217821086EA
:101B2000118681E0838395828482F4018081918192
:101B3000EC8DFD8D9183808320E030E008C026E0AD
:101B400030E005C028E030E002C022E030E0C9010A
:101B50006D96E2E10C94E314C201B1010E945A03B4
:101B6000882309F08ECFEECFC0901001D0901101E4
:101B7000F601848595851C8A1B8A1E8A1D8AA0E031
:101B8000B0E08F8B988FA98FBA8F188A1F86DA8A58
:101B9000C98AF3018081882309F04ACD2ACE80E2E8
:101BA000F50111928A95E9F7D501FE0131968BE096
:101BB00001900D928150E1F78C85F5018487FB8DB2
:101BC000F860FB8F64CFFC018AE0809315019FEFE2
:101BD0009EBD0DB407FEFDCF8EB58F3F29F48091D9
:101BE00015018823A9F722C08E3F01F59FEF9EBD06
:101BF0000DB407FEFDCF8EB580839EBD0DB407FEEC
:101C0000FDCF8EB581836250704011F03296EFCFD8
:101C10008FEF8EBD0DB407FEFDCF8EB58FEF8EBD5D
:101C20000DB407FEFDCF8EB581E0089580E00895E4
:101C3000FC0182E3809316018FEF8EBD0DB407FE89
:101C4000FDCF8EB59FEF9EBD0DB407FEFDCF8EB5C7
:101C50008F3F31F0809116018823A9F790E02EC0C4
:101C60006EBD0DB407FEFDCF6D3F11F491E026C0AF
:101C700090E080818EBD0DB407FEFDCF81818EBDC9
:101C80000DB407FEFDCF915011F03296F2CF8FEFD9
:101C90008EBD0DB407FEFDCF8FEF8EBD0DB407FED8
:101CA000FDCF8FEF8EBD0DB407FEFDCF8EB590E05A
:101CB0008F71853009F091E081E09827892F089590
:101CC000282F82E3809316018FEF8EBD0DB407FE9F
:101CD000FDCF8EB59FEF9EBD0DB407FEFDCF8EB537
:101CE0008F3F31F0809116018823A9F78FEF089577
:101CF0002EBD0DB407FEFDCF872F9927AA27BB273E
:101D00008EBD0DB407FEFDCFCB01AA27BB278EBD2C
:101D10000DB407FEFDCFBB27A72F962F852F8EBDB5
:101D20000DB407FEFDCF4EBD0DB407FEFDCF203430
:101D300011F485E905C0283411F487E801C080E07A
:101D40008EBD0DB407FEFDCF2C3431F48FEF8EBD68
:101D50000DB407FEFDCF8EB59AE02FEF2EBD0DB46A
:101D600007FEFDCF8EB587FF02C09150B9F70895E9
:101D7000A4E0B0E0EEEBFEE00C94D314882311F065
:101D800081E0CFC080910B0181FDC9C08AE09FEF47
:101D90009EBD0DB407FEFDCF2EB58150C9F72A9820
:101DA00040E050E060E070E080E40E94600E81302E
:101DB00009F0A0C084E6809315014AEA51E060E092
:101DC00070E088E40E94600E813009F054C07E010A
:101DD0000894E11CF11C87019FEF9E012B5F3F4F90
:101DE0009EBD0DB407FEFDCF8EB5F80181938F0126
:101DF000E217F307A9F78B81813009F07BC08C8152
:101E00008A3A09F077C040E050E060E070E087E790
:101E10000E94600E823048F440E050E060E070E4E0
:101E200089E60E94600E882321F0809115018823A5
:101E300051F780911501882309F45CC040E050E01F
:101E400060E070E08AE70E94600E882309F052C0CB
:101E50009FEF9EBD0DB407FEFDCF8EB5F7018193B8
:101E60007F01E017F107A9F7898186FD02C012E022
:101E700042C016E040C040E050E060E070E087E71C
:101E80000E94600E823058F440E050E060E070E064
:101E900089E60E94600E823010F412E001C011E069
:101EA000123079F440E050E060E070E087E70E9493
:101EB000600E823078F440E050E060E070E089E647
:101EC00005C040E050E060E070E081E40E94600EF8
:101ED000882321F080911501882311F78091150145
:101EE000882341F040E052E060E070E080E50E942D
:101EF000600E811110E0109317012A9A8FEF8EBDAA
:101F00000DB407FEFDCF8EB5112321F080910B019A
:101F10008E7F03C080910B01816080930B018091C3
:101F20000B012496E6E00C94EF14882311F081E075
:101F3000089580910B0108950F93CF93DF93EB01E8
:101F4000882309F051C0002309F44EC080910B0191
:101F500080FF03C023E030E049C08091170182FD7B
:101F600007C069E0220F331F441F551F6A95D1F740
:101F70002A98013089F4BA01A90181E50E94600E16
:101F8000882321F560E072E0CE010E94E30D00E0BD
:101F90008823E1F401E01AC0BA01A90182E50E9498
:101FA000600E882399F460E072E0CE010E94E30D98
:101FB000882329F0015019F0C050DE4FF4CF40E0E3
:101FC00050E060E070E08CE40E94600E2A9A8FEF8F
:101FD0008EBD0DB407FEFDCF8EB520E030E00023AE
:101FE00029F021E030E002C024E030E0C901DF91B7
:101FF000CF910F910895CF92DF92EF92FF920F93BE
:10200000CF93DF93EB0169017A01882309F064C063
:10201000002309F461C080910B0180FF03C023E01D
:1020200030E05CC080910B0182FF03C022E030E011
:1020300055C08091170182FD07C079E0CC0CDD1CF2
:10204000EE1CFF1C7A95D1F72A98013069F4B7018C
:10205000A60188E50E94600E882381F56EEFCE010F
:102060000E94180E00E027C081FF0EC040E050E043
:1020700060E070E087E70E94600E402F50E060E073
:1020800070E087E50E94600EB701A60189E50E9415
:10209000600E882399F46CEFCE010E94180E8823FD
:1020A00029F0015019F0C050DE4FF5CF6DEF80E000
:1020B00090E00E94180E882309F401E02A9A8FEF1D
:1020C0008EBD0DB407FEFDCF8EB520E030E00023BD
:1020D00029F021E030E002C024E030E0C901DF91C6
:1020E000CF910F91FF90EF90DF90CF900895A0E1F6
:1020F000B0E0EDE7F0E10C94D5148A01882319F0E3
:1021000024E030E0E7C02A98633009F47FC06430EF
:1021100028F4613079F0623051F472C06B3009F408
:1021200096C06C3009F4AAC06A3009F486C024E075
:1021300030E0C6C040E050E060E070E089E40E941A
:10214000600E882309F0B7C060E170E0CE0101960F
:102150000E94E30D882309F4AEC08981829586959B
:10216000869583707A8549858130B1F4872F90E018
:102170000196342F20E0820F931FA0E0B0E02AE008
:10218000880F991FAA1FBB1F2A95D1F7F8018083DA
:102190009183A283B38392C042954695469543703E
:1021A000288530E0220F331F220F331F240F311DEB
:1021B0002F5F3F4F8F8190E083709070982F88271A
:1021C000990F990F280F391F40E050E08E818F70D2
:1021D0006B85661F6627661F860F8E5F7370770F8D
:1021E000870F90E0099704C0220F331F441F551F2B
:1021F0008A95D2F7F80120833183428353835EC0EE
:1022000080E092E0FA019183808358C082E380935A
:1022100016018FEF8EBD0DB407FEFDCF8EB59FEF7B
:102220009EBD0DB407FEFDCF8EB58F3F09F446C0AD
:10223000809116018823A1F73EC080910B0180FD9B
:1022400047C040E050E060E070E089E409C0809160
:102250000B0180FD3DC040E050E060E070E08AE4AA
:102260000E94600E882339F560E170E0C8010E9489
:10227000E30D20E030E0882319F51DC080910B01AB
:1022800080FD26C040E050E060E070E08AE70E94F8
:10229000600E882381F4F8019FEF98012D5F3F4F76
:1022A0009EBD0DB407FEFDCF8EB58083E217F30708
:1022B00029F03196F5CF21E030E002C020E030E097
:1022C0002A9A8FEF8EBD0DB407FEFDCF8EB502C0EA
:1022D00023E030E0C9016096E4E00C94F1148091B1
:1022E0001501882319F08150809315018091160102
:1022F000882319F08150809316019091140183B1C5
:10230000817080931401981749F480910B0190FF1C
:1023100002C0836001C08D7F80930B010895FB0193
:10232000DC0105900D920020E1F70895FB01DC012E
:1023300004C08D910190801921F441505040C8F79C
:10234000881B990B0895FB01DC0102C001900D92DE
:1023500041505040D8F70895DC0101C06D934150C1
:102360005040E0F70895FB019F01E8944230C4F02B
:102370004532B4F44A3029F497FB1EF490958195C8
:102380009F4F642F77270E94FE14805D8A330CF0E4
:10239000895D8193CB010097A1F716F45DE251931B
:1023A0001082C9010C94EC13AEE0B0E0EAEDF1E16B
:1023B0000C94D5140D891E8986E08C831A830983B9
:1023C0008FEF9FE79E838D83CE014996AC016F8985
:1023D000788DCE0101960E94F7112F813885020F6A
:1023E000131FF80110822E96E4E00C94F114ABE078
:1023F000B0E0EDEFF1E10C94C7143C012B015A0160
:10240000FC0117821682838181FD03C06FEF7FEF8D
:10241000C8C19AE0892E1E010894211C311CF301C9
:102420002381F20123FD859123FF81912F018823D0
:1024300009F4B4C1853239F423FD859123FF8191DC
:102440002F01853229F4B30190E00E94FC13E7CFFD
:10245000982FDD24CC249924FFE1FD15D0F09B3288
:1024600069F09C3228F4903259F0933291F40EC006
:102470009D3249F0903369F441E024C052E0D52AFE
:1024800084E0D82A28C098E0D92A25C0E0E1DE2AD5
:1024900022C0D7FC29C0892F80538A3070F4D6FE21
:1024A00005C0989C902C1124980E15C0C89CC02C77
:1024B0001124C80EF0E2DF2A0EC09E3229F4D6FCA9
:1024C0006DC140E4D42A07C09C3619F450E8D52ADF
:1024D00002C0983649F4F20123FD959123FF9191B2
:1024E0002F01992309F0B8CF892F8554833018F034
:1024F0008052833038F444E050E0A40EB51E5FE310
:1025000059830FC0933631F0933779F0933509F042
:1025100056C020C0F5018081898342E050E0A40EBE
:10252000B51E710101E010E012C0F501E080F180FC
:10253000D6FC03C06FEF7FEF02C0692D70E042E070
:1025400050E0A40EB51EC7010E94E1138C015FE7A5
:10255000D52214C0F501E080F180D6FC03C06FEFF6
:102560007FEF02C0692D70E042E050E0A40EB51E7E
:10257000C7010E94D6138C0150E8D52AD3FE07C0AC
:102580001AC0B30180E290E00E94FC13CA948C2D23
:1025900090E008171907A8F30EC0F701D7FC859142
:1025A000D7FE81917F01B30190E00E94FC13C1101E
:1025B000CA94015010400115110579F7ECC094360A
:1025C00011F0993671F5D7FE08C0F501E080F18071
:1025D0000281138144E050E00AC0F50180819181BD
:1025E0007C010027F7FC0095102F42E050E0A40E7C
:1025F000B51E5FE6D52217FF0AC010950095F0942E
:10260000E094E11CF11C011D111D80E8D82A2AE08C
:1026100030E0A101C801B7010E942814F82EF21879
:1026200040C0953729F41D2D1F7E2AE030E01DC0E3
:102630001D2D197F9F3661F0903720F4983509F0F1
:10264000ADC00FC0903739F0983709F0A7C004C06B
:1026500028E030E00AC0106114FD146020E130E091
:1026600004C014FD166020E132E017FF08C0F50138
:10267000608171818281938144E050E008C0F5015E
:1026800080819181BC0180E090E042E050E0A40EA6
:10269000B51EA1010E942814F82EF2188FE7D82E3B
:1026A000D122D6FE0BC05EEFD522F91438F4D4FE49
:1026B00007C0D2FC05C08FEED82202C01F2D01C07A
:1026C000192DD4FE0DC0FE01EF0DF11D8081803368
:1026D00019F499EED92208C01F5FD2FE05C003C0CD
:1026E0008D2D867809F01F5F0D2DD3FC14C0D0FE10
:1026F0000FC01C1510F09F2C0BC09F2C9C0C911A26
:102700001C2D06C0B30180E290E00E94FC131F5F05
:102710001C15C0F304C01C1510F4C11A01C0CC2450
:1027200004FF10C0B30180E390E00E94FC1302FF9D
:102730001EC001FD03C088E790E002C088E590E07C
:10274000B3010CC0802F867891F001FF02C08BE2AC
:1027500001C080E2D7FC8DE2B30190E00E94FC133F
:1027600006C0B30180E390E00E94FC139A94F91430
:10277000C0F3FA94F101EF0DF11DB301808190E0F7
:102780000E94FC13FF20A9F706C0B30180E290E08D
:102790000E94FC13CA94CC20C1F741CEF30166819C
:1027A0007781CB012B96E2E10C94E314FC010590B8
:1027B000615070400110D8F7809590958E0F9F1F43
:1027C0000895FC016150704001900110D8F7809588
:1027D00090958E0F9F1F0895DC01FC01672F71916A
:1027E0007723E1F7329704C07C916D9370836291F7
:1027F000AE17BF07C8F308950F931F93CF93DF93CE
:102800008C01EB018B8181FF1BC082FF0DC02E81EB
:102810003F818C819D812817390764F4E881F98113
:102820000193F983E88306C0E885F985802F09952F
:10283000892B31F48E819F8101969F838E8302C004
:102840000FEF1FEFC801DF91CF911F910F910895F6
:10285000FA01AA27283051F1203181F1E8946F93D1
:102860006E7F6E5F7F4F8F4F9F4FAF4FB1E03ED077
:10287000B4E03CD0670F781F891F9A1FA11D680F15
:10288000791F8A1F911DA11D6A0F711D811D911D48
:10289000A11D20D009F468943F912AE0269F1124BD
:1028A0003019305D3193DEF6CF010895462F477021
:1028B000405D4193B3E00FD0C9F7F6CF462F4F707C
:1028C000405D4A3318F0495D31FD4052419302D0DA
:1028D000A9F7EACFB4E0A695979587957795679580
:1028E000BA95C9F700976105710508959B01AC0180
:1028F0000A2E06945795479537952795BA95C9F7A7
:10290000620F731F841F951FA01D0895629FD00141
:10291000739FF001829FE00DF11D649FE00DF11D9A
:10292000929FF00D839FF00D749FF00D659FF00D49
:102930009927729FB00DE11DF91F639FB00DE11D36
:10294000F91FBD01CF0111240895A1E21A2EAA1B7F
:10295000BB1BFD010DC0AA1FBB1FEE1FFF1FA2174F
:10296000B307E407F50720F0A21BB30BE40BF50B4C
:10297000661F771F881F991F1A9469F760957095D5
:10298000809590959B01AC01BD01CF0108952F92D8
:102990003F924F925F926F927F928F929F92AF92EF
:1029A000BF92CF92DF92EF92FF920F931F93CF933C
:1029B000DF93CDB7DEB7CA1BDB0B0FB6F894DEBFD3
:1029C0000FBECDBF09942A88398848885F846E84F9
:1029D0007D848C849B84AA84B984C884DF80EE8043
:1029E000FD800C811B81AA81B981CE0FD11D0FB64C
:1029F000F894DEBF0FBECDBFED010895AA1BBB1B2F
:102A000051E107C0AA1FBB1FA617B70710F0A61BEE
:102A1000B70B881F991F5A95A9F780959095BC010F
:082A2000CD010895F894FFCFE9
:0C2A280025642C25640A0046415400017E
:00000001FF
